:020000040000FA
:0400000043EF0AF0D0
:08000800AFEF0BF057515A6FE6
:100010005651586F596BD890583759375837593708
:1000200058375937583759373E0E5827000E59233D
:10003000000EFB6EFB225951FA6E5851F96E000EFC
:10004000F86E000EF76E7C0EF66E35EF00F0000EC7
:10005000F86E000EF76E860EF66E35EF00F0000EAD
:10006000F86E000EF76E980EF66E5A51F626D8B05E
:10007000F72AD8B0F82A0800F5501200020202024E
:100080000101020000000101020100000000000067
:100090000000000000000000000002030301020352
:1000A00003030303020203010000FF53D8A45AEF25
:1000B00000F01200F90E0000000000000000000037
:1000C0000000000000000000000000000000000030
:1000D0000000000000000000000000000000FF0F12
:1000E000D8A45BEF00F0000000000000000000005A
:1000F0000000000000000000000000000000000000
:1001000000000000000000000000000000000000EF
:10011000FF2F5AEF00F012000001ED6BEB6B6896B9
:10012000689668966896E251EA6EE151E96EE75189
:1001300001015C6F5C375C35FC0BE926880EEF6EC5
:100140000001E151E96EE85101015C6F5C375C35FB
:10015000FC0BE926080EEF6E0001E151E96EE95152
:1001600001015C6F5C375C35FC0BE926880EEF6E95
:100170000001E151E96EEA5101015C6F5C375C35C9
:10018000FC0BE926080EEF6E6E6A686A050E696E52
:10019000160E706E1E0E716E010E0001F26FEC6F86
:1001A0001200689469946D920001EB6B12000001DB
:1001B000F451F56501D006D0F551F45D80080101D8
:1001C000566F1200F551F45D800F0101566F120059
:1001D0000001F9B1FDD7F29E0601060EEA6E000E8F
:1001E000E96E7F0E0001F4150101596F0001F42B37
:1001F00001015951E9265751EF6E9D880001F551D3
:10020000F4190101586F7F0E581502E10001F981C0
:10021000F28E12000001FC510101566F0F0E5115B4
:10022000576F06EC00F0556FD7EC00F05551566152
:1002300003D0010E566F1200010E556101D004D09B
:100240005251576FE8EC00F0020E0101556101D0E8
:1002500004D05351576FE8EC00F0030E01015561D3
:1002600001D004D05451576FE8EC00F00101566BF7
:1002700012000001E251EA6EE151E96EE95101011B
:100280004D6F4D374D35FC0BE926EFBE96D0000182
:10029000E251EA6EE151E96EE95101014E6F4E37CC
:1002A0004E35FC0BE926E92A040EEF6001D085D01B
:1002B0000001E251EA6EE151E96EE9510101516F2D
:1002C00051375135FC0BE926EC500B6F0C6B0B5181
:1002D0000C6114D00501050EEA6E800EE96E010175
:1002E0000C51E926EF50516F010EEA6E0D0EE96ECA
:1002F0000C51E9265151EF6E0C2BE9D70001E25168
:10030000EA6EE151E96EE9510101516F5137513502
:10031000FC0BE926400EEF160001E151E96EE951B0
:100320000101516F51375135FC0BE926400EEF1A90
:100330000001E151E96EE9510101516F5137513529
:10034000FC0BE926880EEF120C6B0B510C6124D0CC
:10035000010EEA6E0D0EE96E0C51E926EF50516F59
:100360000D0EE96E0C29E926EF50526F0D0EE96E65
:10037000020E0C25E926EF50536F0D0EE96E030EA9
:100380000C25E926EF50546F0AEC01F05653E0E1DA
:10039000040E0C250C6FD9D70001E251EA6EE15131
:1003A000E96EE9510101506F50375035FC0B4F6F2A
:1003B0004F51E926EC50516F1200516B12000101B0
:1003C0000F6B0001F35101010F611ED00001E051DC
:1003D000DE5D02E1DF51DD5D17E2DE51EA6EDD51E7
:1003E000E96EEF500101106F0501050EEA6E400E37
:1003F000E96E01010F51E9261051EF6E0001DD4B4E
:10040000DE2B01010F2BDDD70001F35101010F613C
:1004100002D00001EF6B0001E251EA6EE151E96E9A
:10042000E8510101106F10371035FC0BE926E92A5D
:100430000F51EF6E0001E151E96EE8510101106FBB
:1004400010371035FC0BE926400EEF160001E15184
:10045000E96EE8510101106F10371035FC0BE926E9
:10046000400EEF1A0001E151E96EE8510101106FF1
:1004700010371035FC0BE926880EEF121200000130
:10048000F651F76501D005D0F751F65D01010E6F09
:100490001200F751F65D01010D6F0D1D0E6F0E2B51
:1004A00012000001F751F66303D001010E6B120038
:1004B0000601060EEA6E800EE96E7F0E0001F7154A
:1004C00001010D6F0001F72B01010D51E926EF50DD
:1004D0000E6F1200689A1200698469986D82010E8D
:1004E0000001EB6F1200936A0001E251EA6EE151E4
:1004F000E96EEA510101136F13371335FC0BE9263E
:10050000EFBE5BD00001E251EA6EE151E96EEA51C3
:100510000101166F16371635FC0BE926E92A0F5133
:10052000EF6E126B0F51126113D01151EA6E105120
:100530001225E96EEF50166F0501050EEA6EC00E2A
:10054000E96E01011251E9261651EF6E122BEAD71E
:100550000001E251EA6EE151E96EEA510101166FC4
:1005600016371635FC0BE926400EEF160001E15157
:10057000E96EEA510101166F16371635FC0BE926B4
:10058000400EEF1A0001E151E96EEA510101166FC8
:1005900016371635FC0BE926880EEF120001E151E3
:1005A000E96EEA510101156F15371535FC0B146F13
:1005B0001451E926EC50166F1200166B12006C50A5
:1005C0000001F06FF05101010A6F0A330A330A315A
:1005D0001F0B0B6FD8900B350001F16F040EF01557
:1005E00001010A6F0A330A313F0B0001F125F16F57
:1005F000E251EA6EE151E96EF15101010A6F0A37E9
:100600000A35FC0BE926EF500001C56FE151E96E98
:10061000F15101010A6F0A370A35FC0BE926EC504B
:100620000001C66FE151E96EF15101010A6F0A370D
:100630000A35FC0BE926020EE926EF500001C76FD0
:10064000EC50C86F68963C0EC5150101076F240E6B
:1006500007630DD0040E0001F06306D0060EEF63B1
:100660001200DFEC01F012000C0EF06312003C0EE1
:100670000001C5150101086F040E086313D00001C5
:10068000F053D8B41200080EF0631200030EF215F6
:1006900001010A6F030E0A63120039EC01F0515395
:1006A000FCE012003C0E0001C5150101096F340E7B
:1006B000096312000001E251EA6EE151E96EE7516F
:1006C00001010C6F0C370C35FC0BE926020EE926F4
:1006D000EF500D6FEC500E6F0D510001E56F0101F1
:1006E0000E510001E66FE651EA6EE551E96EEF50FA
:1006F000556EE551E96EEC50566EE551E96E020E0D
:10070000E926EF50576EEC50586EE551E96E040E35
:10071000E926EF50596EEC505A6EE551E96E060E1F
:10072000E926EF505B6EEC505C6E6A90E251EA6E27
:10073000E151E96EE75101010C6F0C370C35FC0BF0
:10074000E926E92A400EEF6E210E55620FD0000116
:10075000E251EA6EE151E96EE75101010C6F0C378D
:100760000C35FC0BE926C80EEF6E0ED00001E251ED
:10077000EA6EE151E96EE75101010C6F0C370C355F
:10078000FC0BE926880EEF6E0001E251EA6EE151A2
:10079000E96EE85101010C6F0C370C35FC0BE926B2
:1007A000080EEF6E6D980001EF6B555215E0550481
:1007B000D8B4CAD0020E556201D000D1800E556265
:1007C00001D0E0D1810E556201D099D3820E5562DD
:1007D0004FEF08F014EF08F056040CE0030E5662D9
:1007E00001D02DD0050E566201D053D0090E5662AD
:1007F000A9D077D0010E576220D058501EE1EC935B
:10080000E251EA6EE151E96EE85101010C6F0C37DB
:100810000C35FC0BE926E92A000EEF6E0001E151D0
:10082000E96EE85101010C6F0C370C35FC0BE92621
:10083000C80EEF6E0001EF6B12007080120057506F
:1008400001010A6F0B6B010E0A6321D00B511FE1EE
:100850000001EC83E251EA6EE151E96EE8510101D9
:100860000C6F0C370C35FC0BE926E92A000EEF6EF5
:100870000001E151E96EE85101010C6F0C370C35B4
:10088000FC0BE926C80EEF6E0001EF6B12007080C2
:1008900012005750EE6F800EEE6121D0E251EA6EE9
:1008A000E151E96EE85101010C6F0C370C35FC0B7E
:1008B000E926E92A000EEF6E0001E151E96EE851E8
:1008C00001010C6F0C370C35FC0BE926C80EEF6EDE
:1008D0000001EF6B050EEF6F090E696E120070805C
:1008E0001200010E5764586602D05750ED6F5752F0
:1008F00005E1585203E1020EF26F02D0030EF26FCF
:10090000E251EA6EE151E96EE85101010C6F0C37DA
:100910000C35FC0BE926E92A000EEF6E0001E151CF
:10092000E96EE85101010C6F0C370C35FC0BE92620
:10093000C80EEF6E0001EF6B480E04010C6F1E0E27
:10094000716E1200708012000B0E566201D006D03C
:10095000560432E0030E56622FD02ED0030EF263FF
:1009600029D059500101046F000EEA6E5D0EE96E48
:100970000451E9265750EF6E0001E251EA6EE15151
:10098000E96EE85101010C6F0C370C35FC0BE926C0
:10099000E92A000EEF6E0001E151E96EE851010114
:1009A0000C6F0C370C35FC0BE926C80EEF6E0001FE
:1009B000EF6B12007080120070801200560404E089
:1009C000030E5662DDD06DD00F0E0101016F700E67
:1009D000006F0F0E5914036F575261E158525FE1D7
:1009E000030E0001F21501010C6F020E0C6326D0FC
:1009F000035324E10151EA6E00510325E96EEF90A3
:100A00000001E251EA6EE151E96EE85101010E6F19
:100A10000E370E35FC0BE926E92A000EEF6E0001B9
:100A2000E151E96EE85101010E6F0E370E35FC0BF6
:100A3000E926C80EEF6E0001EF6B1200030E0001F5
:100A4000F21501010D6F030E0D6327D0030E036134
:100A500024D00151EA6E00510325E96EEF900001A8
:100A6000E251EA6EE151E96EE85101010E6F0E3775
:100A70000E35FC0BE926E92A000EEF6E0001E1516C
:100A8000E96EE85101010E6F0E370E35FC0BE926B9
:100A9000C80EEF6E0001EF6B1200708012007080C4
:100AA00012000F0E01010C6F700E006F0C51016FE0
:100AB0000F0E5914036F575261E158525FE1030E54
:100AC0000001F21501010C6F020E0C6326D00353D6
:100AD00024E10151EA6E00510325E96EEF80000127
:100AE000E251EA6EE151E96EE85101010E6F0E37F5
:100AF0000E35FC0BE926E92A000EEF6E0001E151EC
:100B0000E96EE85101010E6F0E370E35FC0BE92638
:100B1000C80EEF6E0001EF6B1200030E0001F2151C
:100B200001010D6F030E0D6327D0030E036124D066
:100B30000151EA6E00510325E96EEF800001E25198
:100B4000EA6EE151E96EE85101010E6F0E370E3584
:100B5000FC0BE926E92A000EEF6E0001E151E96E77
:100B6000E85101010E6F0E370E35FC0BE926C80E59
:100B7000EF6E0001EF6B12007080120070801200A7
:100B800070801200080E566201D008D0060E566220
:100B900001D023D05652D8B492D11200ED510501A4
:100BA000406F0001E251EA6EE151E96EE851010146
:100BB0000C6F0C370C35FC0BE926E92A010EEF6EA1
:100BC0000001E151E96EE85101010C6F0C370C3561
:100BD000FC0BE926C80EEF6E120058500101056F9C
:100BE000050541E1060E0001EF6F000E01010D6FDA
:100BF0003B0E0001DD6F01010D510001DE6F000EA3
:100C000001010E6F3B0E0D6F106B120E0D250F6F55
:100C10000E5110230F510001DF6F0101105100012F
:100C2000E06FDD51DF5D01010C6F0001DE51E05925
:100C30005C5C03E101010C515B5C12E25B50000162
:100C4000DD2501010D6F5C500E6F0001DE510101C9
:100C50000E230D510001DF6F01010E510001E06F05
:100C6000DFEC01F01200020E056341D0060E000118
:100C7000EF6F000E01010D6F600E0001DD6F0101CD
:100C80000D510001DE6F000E01010E6F600E0D6F41
:100C9000106B650E0D250F6F0E5110230F510001C3
:100CA000DF6F010110510001E06FDD51DF5D0101D7
:100CB0000C6F0001DE51E0595C5C03E101010C5155
:100CC0005B5C12E25B500001DD2501010D6F5C50A1
:100CD0000E6F0001DE5101010E230D510001DF6F87
:100CE00001010E510001E06FDFEC01F01200030E74
:100CF0000563D6D05750066F060E0001EF6F010155
:100D0000065306E0060543E0020E0663BAD07CD027
:100D1000000E0F6FC90E0001DD6F01010F510001C0
:100D2000DE6F000E0101106FC90E0F6F126B000114
:100D3000C95101010F25116F1051122311510001EA
:100D4000DF6F010112510001E06FDD51DF5D010134
:100D50000C6F0001DE51E0595C5C03E101010C51B4
:100D60005B5C12E25B500001DD2501010F6F5C50FE
:100D7000106F0001DE51010110230F510001DF6FE0
:100D8000010110510001E06FDFEC01F01200000ED4
:100D90000F6F290E0001DD6F01010F510001DE6FA1
:100DA000000E0101106F290E0F6F126B29500F25D5
:100DB000116F1051122311510001DF6F0101125107
:100DC0000001E06FDD51DF5D01010D6F0001DE51BB
:100DD000E0595C5C03E101010D515B5C12E25B5088
:100DE0000001DD2501010F6F5C50106F0001DE5125
:100DF000010110230F510001DF6F010110510001AB
:100E0000E06FDFEC01F01200000E0F6F050E000125
:100E1000DD6F01010F510001DE6F000E0101106F47
:100E2000050E0F6F126B05500F25116F1051122315
:100E300011510001DF6F010112510001E06FDD511E
:100E4000DF5D01010E6F0001DE51E0595C5C03E1E2
:100E500001010E515B5C12E25B500001DD250101D6
:100E60000F6F5C50106F0001DE51010110230F5114
:100E70000001DF6F010110510001E06FDFEC01F0B4
:100E800012000001E251EA6EE151E96EE851010100
:100E90000F6F0F370F35FC0BE926CC0EEF6E1200EB
:100EA0000001E251EA6EE151E96EE85101010C6F77
:100EB0000C370C35FC0BE926CC0EEF6E1200EC5112
:100EC0000501406F416B0001E251EA6EE151E96EAC
:100ED000E85101010C6F0C370C35FC0BE926E92AAF
:100EE000020EEF6E0001E151E96EE85101010C6F55
:100EF0000C370C35FC0BE926C80EEF6E12000A0EFB
:100F0000566201D006D0565236E0060E56621200E6
:100F100086D059500101046F030E0001F26329D0FD
:100F2000010E0101046125D0000EEA6E5D0EE96E2E
:100F30000451E926EF500501406F0001E251EA6ECD
:100F4000E151E96EE85101010C6F0C370C35FC0BD7
:100F5000E926E92A010EEF6E0001E151E96EE85140
:100F600001010C6F0C370C35FC0BE926C80EEF6E37
:100F70001200708012000501416B0001E251EA6E1F
:100F8000E151E96EE85101010C6F0C370C35FC0B97
:100F9000E926E92A020EEF6E5950046F020E000195
:100FA000F2631BD00101045318E1000EEA6E5D0EDE
:100FB000E96E0451E926EF500501406F0001E2514E
:100FC000EA6EE151E96EE85101010C6F0C370C3506
:100FD000FC0BE926C80EEF6E1200030E0001F2634F
:100FE0001CD0010E0101046118D0000EEA6E5D0EE6
:100FF000E96E0451E926EF500501406F0001E2510E
:10100000EA6EE151E96EE85101010C6F0C370C35C5
:10101000FC0BE926C80EEF6E1200708012005850CB
:101020000101026F708012005652D8A412000F0EF8
:1010300001010C6F700E006F0C51016F0F0E5914EF
:10104000036F0501416B0001E251EA6EE151E96E67
:10105000E85101010C6F0C370C35FC0BE926E92A2D
:10106000020EEF6E030E036118D00151EA6E0051BB
:101070000325E96E010EEF140501406F0001E251F6
:10108000EA6EE151E96EE85101010C6F0C370C3545
:10109000FC0BE926C80EEF6E120070801200708003
:1010A00012006AA005D06BA003D00001CD4BCE2B5F
:1010B0006AA205D06BA203D00001CF4BD02B6AA44B
:1010C00005D06BA403D00001D14BD22B6AA605D06A
:1010D0006BA603D00001D34BD42B6AA805D06BA814
:1010E00003D00001D54BD62B6AAE05D06BAE03D032
:1010F0000001DB4BDC2B6A6A689212000001F9B335
:1011000003D0FD6BFE6BF983E251EA6EE151E96EAB
:10111000EA5101010C6F0C370C35FC0BE926EFBED0
:1011200012003FEC02F00E510001FE6FD8B4120025
:1011300051EC02F00E510001FD6FFDAF8ED0F80EA4
:10114000FD616BD0FD51516EFA510101566F0001E6
:10115000FD390F0B01010D6F070E0D15576F06ECD2
:1011600000F0526E525256E10001FB510101566FE0
:101170000F0E0001FD150101576F06EC00F0526ED5
:10118000F00E0001FD6305D0F00E4E6E010E546EA0
:1011900041D0F70EFD633ED0545203E054040DE0FD
:1011A00019D04D38F00B01010E6F050E0E11086FAE
:1011B000F70E096F0A6B0B6B1AD04D38F00B01015B
:1011C0000E6F060E0E11086F4E50096FF70E0A6F64
:1011D0000B6B0DD04D38F00B01010E6F070E0E1189
:1011E000086F4E50096F4F500A6FF70E0B6F030ECA
:1011F0000001F21501010D6F030E0D630AD0040EFC
:101200000F6F010E116F080E106F73EC02F0165382
:10121000F6E0546A5250536E12004D38F00B010143
:101220000E6F0F0E0E11086F0001FD510101096FC5
:101230000A6B0B6B030E0001F21501010D6F030E1B
:101240000D631200040E0F6F010E116F080E106F68
:1012500073EC02F01653F6E01200F00E516230D03B
:10126000542A540404E0020E546207D003D0FD5106
:101270004E6E1200FD514F6E1200FD51506E4D38F2
:10128000F00B01010E6F040E0E11086F4E50096F26
:101290004F500A6F50500B6F030E0001F215010101
:1012A0000D6F030E0D630AD0040E0F6F010E116F48
:1012B000080E106F73EC02F01653F6E0546A120039
:1012C000535203E15204536E01D05306520404E119
:1012D000FD514F6E506A07D0535203E1FD51506EDD
:1012E00002D0FD514F6E5352D8A41200F00E51148B
:1012F00001010D6FF00E0D6301D008D04D38F00BD9
:101300000F6F51380F0B0F11086F19D0525203E0B5
:10131000520408E00ED04D38F00B0F6F050E0F1180
:10132000086F0DD04D38F00B0F6F020E0F11086FC4
:1013300006D04D38F00B0F6F030E0F11086F515090
:10134000096F4F500A6F50500B6F030E0001F215DA
:1013500001010E6F030E0E631200040E0F6F010EDB
:10136000116F080E106F73EC02F01653F6E01200C6
:10137000F29EAB98AB889D8A9D88F28CF28E12000B
:101380000001F991F76BF66BF56BF46B948E949CFE
:10139000FF5304E0040E0101016F02D00101016B53
:1013A0000051AF6E0151AC6EAC50200FAC6E900E80
:1013B000AB6E4D6A516A526A536A546A120068B63B
:1013C000DFEC02F068BA6AEC02F068B251EC08F0A7
:1013D00069B86CEC02F01200140E6F6E400E000142
:1013E000F36F010E696E686A200EA06E400E6D6E7E
:1013F000080E6D6EED6B010EEC6F0101006B016B61
:10140000026B0001EF6BCD6BCE6BCF6BD06BD16BF2
:10141000D26BD36BD46BD56BD66BDB6BDC6BC00E36
:10142000F210F26E1200936A010E946E580E0001D3
:10143000FF6F55EC00F0010EFF6F2F0E0101006FE2
:10144000C0EC09F0B8EC09F0ECEC09F0DFEC09F0C5
:10145000030E0001F215FF6F030EFF63F7D7545020
:101460000101076F5350066F5250056F5150046FC2
:101470005050036F4F50026F4E50016F4D50006F30
:101480007EEC08F0E3D70001F993E76B010EE86FFB
:10149000020EE96F030EEA6F400E0401016F026B4A
:1014A000050E036F056B400E066F050E076F400EAD
:1014B000096F800E0A6F050E0B6F0D6BC00E0E6F5D
:1014C000050E0F6F0001CD6BCE6BCF6BD06BD16B68
:1014D000D26BD36BD46BD56BD66BD76BD86BD96B08
:1014E000DA6BDB6BDC6BF46BF56BF66BF76BF86B45
:1014F000E36B040EE46FE351E16FE451E26F000E21
:10150000FA6F010EFB6F020EFC6F040EC96F030E23
:10151000CA6F090ECB6F040ECC6F120E296E030E2C
:101520002A6E4D0E2B6E2C6A650E2D6E2E6A670E7E
:101530002F6E306A610E316E326A440E336E346A39
:10154000720E356E366A750E376E386A6D0E396EEC
:101550003A6A240E056E030E066E4D0E076E086A7B
:10156000650E096E0A6A670E0B6E0C6A610E0D6ECF
:101570000E6A440E0F6E106A720E116E126A750EAC
:10158000136E146A6D0E156E166A200E176E186AA9
:101590004D0E196E1A6A490E1B6E1C6A440E1D6EA2
:1015A0001E6A490E1F6E206A200E216E226A550E99
:1015B000236E246A530E256E266A420E276E286A11
:1015C000120E3B6E010E3C6E3D6A020E3E6E3F6A8D
:1015D000406A416A400E426ED80E436E040E446E5D
:1015E0000A0E456E466A476A010E486E010E496E44
:1015F000020E4A6E4B6A010E4C6E090E606F020EAF
:10160000616F650E626F636B020E646F010E656F32
:10161000666B800E676F320E686F090E696F040E7D
:101620006A6F6B6B6C6B6D6B010E6E6F010E6F6F83
:10163000706B716B090E726F240E736F010E746FF5
:10164000756B010E766F090E776F786B010E796FEF
:10165000010E7A6F090E7B6F040E7C6F010E7D6F99
:101660007E6B020E7F6F010E806F030E816F826BA7
:10167000836B070E846F240E856F010E866F876B58
:10168000010E886F410E896F8A6B060E8B6F240ED8
:101690008C6F020E8D6F010E8E6F010E8F6F906B2F
:1016A000060E916F240E926F020E936F020E946FCE
:1016B000020E956F966B090E976F240E986F030EAE
:1016C000996F010E9A6F030E9B6F010E9C6F020EB5
:1016D0009D6F010E9E6F9F6B090EA06F240EA16F70
:1016E000030EA26F020EA36F040EA46F010EA56F6E
:1016F000010EA66F010EA76FA86B090EA96F050E4C
:10170000AA6F010EAB6F020EAC6F400EAD6FAE6BE9
:10171000AF6BB06BB16B050EB26F250EB36F010EE0
:10172000B46F010EB56F010EB66F090EB76F050EDF
:10173000B86F810EB96F020EBA6F400EBB6FBC6BF3
:10174000BD6BBE6BBF6B050EC06F250EC16F010E6A
:10175000C26F010EC36F030EC46F13EF0AF0EACF1E
:1017600001F0E9CF02F0F4CF03F0F3CF04F09DAA2B
:1017700029D09EAA27D0ABA2ABB46BD0AE5001014A
:101780005B6F5D6B800E0001F72501015C6FD8B0C7
:101790005D2B0001F65101015C6302D05D5159E0FF
:1017A0000601060EEA6E800EE96E7F0E0001F61548
:1017B00001015E6F0001F62B01015E51E9265B51CC
:1017C000EF6E47D09DA81DD09EA81BD00001F451FC
:1017D000F563F46314D00601060EEA6E000EE96E9E
:1017E0007F0E0001F51501015C6F0001F52B010171
:1017F0005C51E926EF50AD6E0001F9912AD09D9819
:1018000028D0A0AA26D0A1AA24D068A404D069A474
:1018100002D0D1EC00F068A004D069A002D08CEC1A
:1018200000F068A615D069A613D0050E0001EF637D
:101830000ED0EF6BED6BEE516E6E010E696E000E09
:10184000EE6503D0020EF26F02D0010EF26F6896C1
:10185000A19A04C0F3FF03C0F4FF02C0E9FF01C076
:04186000EAFF11008A
:020000040030CA
:0E000000320E3F1EFF8085FF0FC00FE00F4045
:00000001FF
